:0200000270008C
:10800000000001205D8307004583070047830700C8
:10801000498307004B8307004D83070000000000E1
:1080200000000000000000000000000015D2070062
:1080300051830700000000005383070055830700A9
:1080400057830700578307005783070057830700AC
:10805000578307005783070057830700578307009C
:10806000578307005783070057830700578307008C
:10807000578307005783070057830700578307007C
:10808000CDB40700578307005783070057830700C5
:1080900057830700578307001DD407005783070045
:1080A000578307005783070057830700578307004C
:1080B00057830700578307000000000000000000FE
:1080C000578307005783070057830700578307002C
:1080D00045B10700578307005783070000000000E1
:1080E0000000000000000000000000000000000090
:1080F0000000000000000000000000000000000080
:10810000000000000000000000000000000000006F
:10811000000000000000000000000000000000005F
:10812000000000000000000000000000000000004F
:10813000000000000000000000000000000000003F
:10814000000000000000000000000000000000002F
:10815000000000000000000000000000000000001F
:10816000000000000000000000000000000000000F
:1081700000000000000000000000000000000000FF
:1081800000000000000000000000000000000000EF
:1081900000000000000000000000000000000000DF
:1081A00000000000000000000000000000000000CF
:1081B00000000000000000000000000000000000BF
:1081C00000000000000000000000000000000000AF
:1081D000000000000000000000000000000000009F
:1081E000000000000000000000000000000000008F
:1081F000000000000000000000000000000000007F
:10820000314932480A1A02D0072291438D4630493B
:1082100030480A1A06D00722914381F309880222C6
:1082200082F314882C482D492D4A00F03CF82D4843
:108230002D492E4A00F037F82D482E492E4A00F0DD
:1082400032F82E482E492F4A00F02DF82E482F499B
:108250002F4A00F028F82F482F49304A00F023F821
:108260002F483049304A00F01EF83048304900228B
:1082700000F024F82F483049002200F01FF82F4A60
:1082800090471F481F49884205D00268043003B454
:10829000904703BCF7E700208646EC46002000210B
:1082A000274A9047FEE7884207D0521A05D0037844
:1082B00001300B700131013AF9D17047884202D088
:1082C00002700130FAE770470000012000F800203A
:1082D000000001200000012080DC07007C59002004
:1082E000B4590020B8830700B88307003ED70700C1
:1082F00080DC07007C5900207C590020ACD70700A7
:10830000ACD70700ACD70700ACD70700ACD7070045
:10831000ACD70700ACD70700ACD7070080DC07005C
:10832000B8DC0700B4590020B4590020B45900202B
:10833000647F0020647F0020647F00208583070025
:10834000319D0700FEE7FEE7FEE7FEE7FEE7FEE7FA
:10835000FEE7FEE7FEE7FEE700F002B8FFF7FCBF2E
:108360000F484FF00701884385460E4880470E4866
:10837000016841F470010160BFF34F8FBFF36F8F4D
:10838000FFF73EBF09480A490A4A884207D0521AF5
:1083900005D0037801300B700131013AF9D17047F3
:1083A000000001208DB5070088ED00E098D7070098
:0883B000685900207C590020EF
:1083B8004B1C30B5DB00044612F003009BB20DD114
:1083C800074D2A601A44074B1A60074B1870074B71
:1083D8001870074B1C80074B198030BD0720FCE73D
:1083E800BC590020B8590020B4590020C4590020B5
:1083F800C0590020C25900202DE9F3472B4F3B8874
:108408008B4206460D4690464BD300240DF10700DB
:108418008DF8074000F086F8254B26481A78264B39
:10842800008893F800C084455FFA8CF138BF4C1C73
:10843800D2B238BFE4B2A2422DD01C781A78D1B299
:10844800904286BF0131C9B2002119709DF807001A
:1084580000F08CF84FF6FF739C4224D0DFF8609050
:10846800D9F800204FEAC40A42F8348002EBC4036A
:10847800A6B19DB1114B38881B682A4604FB003011
:10848800314605F0CCF8D9F80030534400209D80DF
:1084980002B0BDE8F0874FF6FF74D7E70020988058
:1084A800F6E70920F4E70420F2E700BFC0590020EE
:1084B800C4590020C2590020B4590020B8590020DE
:1084C800BC590020F8B5114C114D264622782B785E
:1084D8009A4200D1F8BD0F480F4A237812680788DE
:1084E8000E4802EBC301006852F83320898803FB69
:1084F800070090470A4922780988D3B2914286BF7B
:108508000133DBB200233370E0E700BFC459002019
:10851800B4590020C0590020BC590020B859002087
:10852800C259002070B5EFF3108672B60C4A9468F1
:1085380001239CB993600B4B0B4DD3F88010294055
:108548001160C3F88050D3F8841051604FF0FF32A7
:10855800C3F88420047006B962B670BD0370FAE7E8
:10856800C859002000E100E0FC06FFBD084B9A68EE
:1085780010B55AB150B9EFF3108172B6054A1C68AC
:1085880014605C685460986001B962B610BD00BFA1
:10859800C859002000E100E030B53AB11368DB4368
:1085A8000A4D0144814204D1D84330BD4FF0FF3316
:1085B800F6E710F8012B5340082213F0010418BF06
:1085C8002C46013A84EA5303F7D1EBE72083B8ED50
:1085D80010B561B1B2FBF3F403FB1424A4B244B99F
:1085E800C0E9001484608281C381204610BD0E203A
:1085F800FCE70920FAE782B050E8022FC188B2EB05
:10860800324F4FF0000317BF92B241EA014142EAEC
:10861800014104E04268B2EB324F08BF012340E851
:108628000212002AE8D18DF807309DF80730002B98
:108638000CBF1120002002B0704737B550E8013F49
:108648009DB2C48925448489A54228BF2D1B04896D
:10865800A54202BFBFF32F8F002207E0C5EA03053A
:1086680040E80154002CE9D14FF001028DF80320B5
:108678000193019B9DF803200B6002F0FF0322B1D8
:108688000B880068184403B030BD1846FBE70A8819
:108698004B889A4209D150E8012FC2EA024240E8C9
:1086A8000123002BF7D1012070470020704737B510
:1086B80050E8023F1FFAA3F5C488A54202BFBFF3E2
:1086C8002F8F00220DE0C48925448489A54228BF44
:1086D8002D1BC3EA054540E80254002CE8D14FF0B1
:1086E80001028DF803200193019B9DF803200B6084
:1086F80002F0FF0322B14B880068184403B030BD74
:108708001846FBE70A884B889A4209D150E8022F9D
:10871800C2EA224240E80223002BF7D10120704729
:108728000020704710B5034653E8000F40EA0102E5
:1087380043E8002494F0000FF6D110BD10B50346AD
:1087480053E8002F02EA010043E8000494F0000F08
:10875800F6D110BD0121FFF7E5BF0021FFF7EEBFFD
:1087680010B590B1D0E9012301689B1ADBB20A6009
:10877800013BDBB2FF2B026802D10020107110BD53
:1087880011684C1C14600B70F2E70E20F7E737B540
:10879800054600240DF107008DF80740FFF7C2FEDB
:1087A8002A686B68116899420ED9481E106011F842
:1087B800014CEB68298A01FB0434AB6811791B1A58
:1087C800DBB2994238BF13719DF80700FFF7CEFE60
:1087D800204603B030BD37B5054600230DF107002C
:1087E8000C468DF80730FFF79DFE2A681368591C60
:1087F8001160E968641A298AB4FBF1F41C709DF8C9
:108808000700FFF7B3FE03B030BD0B6801601146E7
:10881800184710B40468E468A4465DF8044B604740
:1088280010B404682469A4465DF8044B604700004E
:1088380070B550B90E4D0F4C0026641B1423B4FBC1
:10884800F3F4B44208D1002010E00368002BF1D003
:10885800BDE87040DB6918472B6813B90136143539
:10886800EFE7DB69284698470028F7D070BD00BFBE
:10887800685900207C590020014B43600020704754
:10888800ACD707000846704700207047024B1868AD
:10889800003818BF01207047D459002008B5024895
:1088A800FFF75BFF002008BDD459002008B510462B
:1088B8001A4604F0B4FE002008BD00002DE9F0437C
:1088C800814687B014480E4615469846FFF742FF82
:1088D8000446F0B90746BD4215D10F48FFF73DFFE2
:1088E800D9F808305BB102228DF800200022CDE9CA
:1088F8000126CDE90325CDF814806846984720461F
:1089080007B0BDE8F08306EB073001F071F80137D6
:10891800E1E71124F3E700BFD45900202DE9F04125
:10892800804686B011480F4616461D46FFF712FFCF
:108938000446C8B9AA083146384601F087F80B48FA
:10894800FFF70BFFD8F8083053B101228DF800204B
:108958000C9A0592CDE90147CDE903656846984729
:10896800204606B0BDE8F0811124F9E7D45900206B
:1089780029DF704728DF704770B503689E6886B0A6
:1089880004460D466EB114220021684604F070FEBC
:10899800A3680593237901952BB1012B0DD0684667
:1089A800B04706B070BD01238DF8003023690293EB
:1089B800E368039363690493F1E702238DF80030B9
:1089C800E3681B030293F5E70846704700207047E9
:1089D800024B187A003818BF01207047C45B00208A
:1089E800034B187A0122B0FA80F05A744009704794
:1089F800C45B002008B510461A4604F010FE00209B
:108A080008BD000008B514220021044804F030FE17
:108A18000348FFF7F0FD002008BD00BFC45B00203D
:108A2800B45B002010B5094C094B43602046FFF7A2
:108A380091FE48B904F0D4FC064920741C2306486A
:108A48004FF4EE72FFF7C4FD002010BDC45B002098
:108A5800D8D70700D8590020B45B002070B5234C44
:108A6800234E237A25463BB922492348FFF71FFEA8
:108A7800306008B9606070BD022334682B722379B6
:108A880073B1012B22D020460321FFF775FF002385
:108A98002B726B6017491848BDE87040FFF732BE6B
:108AA800D4E90523D21A142AD4E9031028BF1422C2
:108AB8009208012A38BF012219441844FFF758FFC9
:108AC80050B11128DFD101232B72D4E7D4E9030375
:108AD8001844FFF74FFFF3E72B7C002BCBD101465F
:108AE800BDE87040022000F009B800BFC45B002058
:108AF800DC5B0020D85B0020B45B002038B5831E07
:108B0800012B43D8224C237A002B3FD0022B09D1CA
:108B180003282ED01F4B00221B68E2601A793AB155
:108B2800012A20D0637C6BBBBDE83840FFF796BFB5
:108B3800D3E905128D1A142D94BF521914329A6173
:108B48009142EFD102284FF0000308BF1946237263
:108B5800104B18BF0D211868FFF70EFF0E490F487C
:108B6800FFF7D0FDDEE71A6901321A615B699A42A4
:108B7800E7E7E3680133082B01D8E360D2E7002375
:108B8800E360DFE7BDE8384004F01ABC38BD00BF39
:108B9800C45B0020DC5B0020D85B0020B45B0020B5
:108BA80000F0FD03012B08D1044B00225A74421E29
:108BB800504250411874FFF751BF7047C45B002002
:108BC80010B5064C201DFFF7C5FD28B9637C1BB9FD
:108BD800BDE81040FFF742BF10BD00BFC45B0020D6
:108BE8002DE9F34180460D460F4801A916461F4658
:108BF800FFF723FD0446A8B11C22002104F038FD2C
:108C08002D0B0123237101A90748C4F80080A76030
:108C1800E5606661FFF73BFDFFF7D2FF002002B079
:108C2800BDE8F0810420FAE7B45B00202DE9F743A2
:108C380081468846104801A917461E46FFF7FDFCE5
:108C48000446B0B11C22002104F012FD00250A9B45
:108C5800A36001A9C4E9037807482571C4F8009006
:108C68006661FFF714FDFFF7ABFF284603B0BDE8C8
:108C7800F0830420FAE700BFB45B00200B684A6861
:108C88004360934208BF0023016008BF43607047F8
:108C9800436843B10268916852680B449342436049
:108CA80004BF0023436070472DE9F04FC9B008AAFC
:108CB80001F1400514464B780E781B0443EA06631D
:108CC800CE7833438E78043143EA06238D4244F844
:108CD800043BF0D11024916B16464FEAF14383EA26
:108CE800714383EA9123716A366852F8045F31440C
:108CF8000B444FEAB54181EAF51181EAD501013407
:108D08000B44402CD363E6D1D0E914E30093836D80
:108D18000193C36D0293036E0393436E0493836EB2
:108D28000593C36E0693DDE9057BDDE9031CDDE9E8
:108D380001592B4B009E079374464FF00008079B80
:108D480053F8042B07934FEAF12383EAB11383EA1C
:108D5800716A08AB53F828301A440AEB020327EA71
:108D6800010A01EA0C028AEA02021A444FEA743A3A
:108D780086EA05035A448AEAB40A06EA050B234040
:108D880083EA0B038AEAB45A08F101089A44B8F155
:108D9800400F02EB0903BB465244A94619D172445D
:108DA8000265009A22444265019A32448265029A19
:108DB8002A44C265039A1A44049B02660B4443661C
:108DC800059B63448366069B3B44C36649B0BDE884
:108DD800F08F674635468C46264619461446AEE758
:108DE80004D8070030B5E0B10F4A10490024002527
:108DF800C0E91245C0E914120D4C0E4A0E4DC0E9E7
:108E080016420E4AC0E918520D4A826602F174529F
:108E1800A2F523020023A2F692420364C266184612
:108E280030BD0E20FCE700BF85AE67BB67E6096A68
:108E380072F36E3C3AF54FA57F520E518C68059B34
:108E4800ABD9831F70B5F0B1DAB900201CE00C462D
:108E58008D180026AC42F8D0036C14F8012BC254CC
:108E68000133402B0364F5D10146FFF71DFFD0E91C
:108E7800123213F5007342F10002C0E9123206649F
:108E8800E8E70029E3D10E2070BD70B50D461646FF
:108E98000446002875D0002973D0026C8021372A37
:108EA800815402F101034FF0000240D8382B39D128
:108EB800D4E91201226C0823E3FB020103BAE3633D
:108EC8000B0A84F83A300B0C84F839300B0EC4E9DD
:108ED800120184F83B1084F8383021462046FFF709
:108EE800E3FE691E76B30023E26EDA4001F8012F33
:108EF800A26EDA400A71626EDA400A72226EDA40B5
:108F08000A73E26DDA400A74A26DDA400A75626D7E
:108F1800DA400A76226DDA400833202B0A77E3D14B
:108F2800002070BDE2540133C0E7E25401333F2B07
:108F3800FBD921462046FFF7B7FE3822002104F06E
:108F480097FBB5E71823226DDA4001F8012F626D0F
:108F5800DA400A71A26DDA400A72E26DDA400A73E9
:108F6800226EDA400A74626EDA400A75A26EDA403E
:108F78000A76E26EDA40083B13F1080F0A77E2D16D
:108F8800CEE70E20CDE743689B68184708B54368CD
:108F980008305A7900F079FE002008BD2DE9F0412B
:108FA8000C469CB008461F460392FFF7ECFFD4F826
:108FB8000480039998F80550BD4228BF3D460646EF
:108FC8002A4604A800F056FE98F8052022990CA815
:108FD80000F05BFE00960CAB2A4604A904F10800D9
:108FE80001F028FD002848F2425018BF00201CB0AC
:108FF800BDE8F0810023C0E902328B881A44B1F938
:10900800063002611A44C0E900114261088800383C
:1090180018BF012070474268118838B503460029F7
:1090280037D0148A02F1100141602CB9C268016876
:10903800FFF7E0FF204638BD9078118900F0300531
:10904800302D14D1947C04F03004302C1BD190883E
:109058001969091A19610021908AB2F91620084481
:10906800196901441961114459610120E3E700F0CD
:10907800F004202C07D150894143002DECD1986889
:1090880001309860E8E700F0C000802808BF04219C
:10909800F3E70846CFE770B5466804460D466368AF
:1090A8001A88AA4204D19B7803F00F03082B07D132
:1090B8002046FFF7B0FF6368B342F0D1002070BDCF
:1090C8000120FCE743681A44426011B101399A4211
:1090D80001D10120704713F8010B01F8010FF6E7E1
:1090E80083682DE9F3410446884623B900263046B3
:1090F80002B0BDE8F081036801220DF1070198472D
:1091080006460028F2D0A3689DF80750013BA360EB
:109118009DF90730002B1ADA05F07F050727A368A9
:10912800002BE3D0236801220DF107012046984760
:109138000028DBD0A3689DF80720013BA36002F05C
:109148007F03BB401D43130607F1070702D4C8F885
:109158000050CCE7232FE2D1C8E770B54568AA785C
:1091680002F00F06082E86B003461FD103691C685B
:1091780000260CB906B070BD236862689D68267326
:1091880029466846FFF736FF6368049304F10C0329
:109198000593AB7803F0C003802B08BF231D6846F6
:1091A80008BF0493FFF7D9FFA468E2E712F0C001F3
:1091B8001CD102F0300010280AD15A691170072E0C
:1091C800EC68186909D10146204600F017F8D1E784
:1091D8009006F4D55B691980CCE72A89214614B139
:1091E80004F01DFAC6E704F043FAC3E78029C1D1A9
:1091F8000069002192060160BCD5EBE77FB50A46FD
:1092080001466846FFF7F6FE30B16846FFF7A5FF4E
:109218006846FFF700FFF7E707B05DF804FB0000BA
:1092280030B5044685B01546A9B90268114B9A4273
:1092380011D0102D06D82A4669462046FFF7F0FFC0
:1092480005B030BD102269462046FFF7E9FF002827
:10925800F6D0103DEDE7A368AB4201D20020EFE75E
:1092680023682A46204698470028F7D0A268521B50
:10927800A260E5E7CD900700F7B50E4601A90746BD
:109288001546FFF72DFFA8B1019A0123D3184FF017
:10929800000404D2B17801F0C001802901D1204630
:1092A80008E031899942FAD329463846FFF7B8FFD2
:1092B800019BEC5403B0F0BD73B50D4601A90646F9
:1092C8001446FFF70DFF98B1019AB2F5803F11D20D
:1092D800AB7803F0C003802B02F102010AD02B897E
:1092E8008B4207D32146304621F8022BFFF798FF1F
:1092F80002B070BD0020FBE710B5034C826000226D
:10930800C0E90041C26010BDCD9007002DE9F341CE
:10931800002604460F46B0463546A3682BB323689B
:1093280001220DF1070120469847F0B1A3689DF886
:1093380007C0013B0CF07F02C5F12001A360A5F135
:10934800200302FA03F322FA01F10B43AA401CF0AE
:10935800800F46EA020643EA080805F1070502D12C
:10936800C7E9006802E0462DD7D1002002B0BDE869
:10937800F08173B50C4669461646FFF7C7FF68B11A
:109388002389082B0CD1DDE90045C6E90045DDE954
:109398000023AB4206BFA2420120002002B070BDEC
:1093A800042B04D1009B33601C460025EFE7022BF9
:1093B8004FF0000004D1009B33809CB20546E6E7DD
:1093C800012BEBD1009B337003F0FF04F6E737B5B0
:1093D8000D4669461446FFF799FF30B12A89082AD5
:1093E800DDE9003103D1C4E9003103B030BD042AFE
:1093F80018464FEAE37108D123601A460B468B42A0
:1094080006BF824201200020EFE7022A04D11BB2E6
:1094180023801AB2D317F2E7012A03D15BB2237073
:109428005AB2F7E70020E0E7F7B51F4600233B7084
:109438000D460B70136001A904461646FFF750FE4F
:1094480030B9A36813B901233B70002003B0F0BD05
:10945800019C002CF7D0E30804F0070433602C705B
:10946800F4E713B5044605291FD8DFE801F0030F18
:10947800151E1E1C012201A92046FFF7D1FE18B1B6
:109488009DF90430002BF5DB02B010BD0822002145
:109498002046FFF7C5FEF7E701A9FFF721FE0028E0
:1094A800F2D0019AF3E70422F1E70020ECE773B564
:1094B8000D4601A90446FFF713FE064618B9002613
:1094C800304602B070BD94E80F0085E80F0001999E
:1094D8008A42F4D3A960A3685B1AA360F0E700008E
:1094E8002DE9F0435668B37813F0C00489B00746F5
:1094F8008C46154603D0402C67D000240CE003F0BE
:109508000F025D4903F03003202B51F8228023D04D
:1095180006D8E3B1102B17D0204609B0BDE8F08378
:10952800302BF9D16B6931881980072A09D1214676
:109538003289286904F09CF86B682969D868FFF7B4
:109548005DFE2A6969683EE06B6901221A702A6922
:109558003146C0470446DFE7BCF1020FD5F8149046
:1095680024D1042A22D804A9FFF7A1FF0446002821
:10957800C3D0069B2BB16968B9F800304A899A4272
:1095880005D8059B7B60069B002BC5D0B5E70889ED
:109598002A6903FB002204A8C04728B1B9F80030A3
:1095A8000133A9F80030E4E70446EAE7B9F80030E7
:1095B80072899A42A1D931892A69581C03FB012270
:1095C800A9F8000031463846C3E7D2F8108046466D
:1095D80056F8043B13B9FFF744FFBBE7022914D13F
:1095E80004A9FFF764FF002887D0D8F8003069681D
:1095F800324604A89847044600283FF47EAF069BED
:10960800002BF2D1059B7B6086E7012925D005292F
:109618002BD000297FF471AF0C460DF104090134F9
:109628000B2C3FF46AAF012249463846FFF7F8FD94
:1096380000283FF462AF19F9013B002BEFDB0F4B19
:10964800049301ABCDE90534002307936968D8F882
:109658000030324604A898477CE7082201A9FFF7A2
:10966800DFFD08240028EAD147E704220DEB0201B8
:10967800FFF7D6FD0424F5E710D90700CD900700C1
:109688002DE9F04F91B00446002604A8CDE9026602
:10969800FFF7B0FCA3683BBBDDE9053404A89D785F
:1096A800FFF7B9FC0028F7D115F0300F03D1059B5F
:1096B8001B8803B10134002C00F0A9806309002243
:1096C80002A9934240F09C8010AA02EB830304F0A5
:1096D8001F0453F8383CC4F120044FF0FF30E04039
:1096E800C31A584258410DE00DF1030301AA0DF1C8
:1096F80002012046FFF798FE38B99DF80330002B89
:10970800CAD1002011B0BDE8F08F019904A8FFF775
:10971800C2FC002850D1019BB3427DD3059D059A18
:10972800937803F00F03082B7FD004A8FFF773FC8E
:10973800059B9D42F3D14FF0FF36019FB7426BD393
:10974800089B9DF802A0D4F808801D684FF0010915
:10975800A368002D5DD098459CD12B68D3F800B044
:10976800BBF1000F08D053463A4629462046D84751
:109778000028C6D0AD68EBE7D3F808B0BBF80030D6
:109788009F42F7D16A6859460AA8FFF733FC6B680D
:109798000E9305F10C030F939BF8023003F0C003FE
:1097A800802B04BF2B1D0E930AAA85F80C905146F6
:1097B8002046FFF795FEDBE7059B9B7813F0300FFB
:1097C8000FD1069A3F2A0CD8510910AB03EB81013F
:1097D80002F01F020123934051F8382C134341F83B
:1097E800383CE5682DB19DF80220019904AB20466C
:1097F800A8479DF8021004AA2046FFF771FE10E062
:1098080051F8225001357FF47DAF013259E701202C
:1098180078E798457FF43EAF9DF802102046FFF7A1
:1098280020FE00287FF436AF6BE7168885E737B54A
:109838000C460546114620460192FFF7DFFC019AC7
:109848002146284603B0BDE83040FFF719BF70B580
:1098580086B0CE6801920C4602A90546FFF727FE9E
:1098680068B1E06858B1A378019A03F03003202B5F
:10987800314602A805D1FFF7DAFF039B6B6006B0FB
:1098880070BDFFF7FDFEF8E7D3B50C466946FFF754
:109898003DFD80B1DDE9001300274A0801F001060B
:1098A80042EAC37256EA07014FEA53031CBFD24388
:1098B800DB43C4E9002302B0D0BD37B50D46694685
:1098C8001446FFF7E1FF68B12B89082B0CD1DDE9BD
:1098D8000001C4E90001DDE900238B4206BF824292
:1098E8000120002003B030BD042B03D10098206074
:1098F800C117F0E7022B04D1BDF90000208000B2A7
:10990800F6E7012B04D19DF90000207040B2EFE783
:109918000020E7E713B504220C460DEB0201FFF720
:109928007FFC08B1019B236002B010BD1146FFF710
:10993800F1BF13B508220C466946FFF771FC18B150
:10994800DDE90023C4E9002302B010BD1146FFF78A
:10995800F0BF0000044B1A5C012393404FF0A04273
:10996800C2F80C35704700BF34D90700044B1A5CA5
:10997800012393404FF0A042C2F80835704700BF5A
:1099880034D9070008B50020FFF7F0FF0120FFF7E2
:10999800EDFF0220FFF7EAFFBDE808400320FFF7CC
:1099A800E5BFC20708B501460CD54FF0A043032216
:1099B800C3F84427C3F84827C3F84C27C3F85027EF
:1099C800FFF7E0FF8B070AD54FF0A0430C22C3F83E
:1099D8003427C3F83827C3F83C27C3F8402708BD05
:1099E800024AD2F80034002BFBD0704700E0014057
:1099F8000A4908B50223C1F80435BFF36F8FBFF3D6
:109A08004F8FC1F80805FFF7EBFF0023C1F80435B5
:109A1800BFF36F8FBFF34F8F08BD00BF00E0014059
:109A280010B5094C0123C4F80435BFF36F8FBFF399
:109A38004F8F0160FFF7D4FF0023C4F80435BFF34C
:109A48006F8FBFF34F8F10BD00E001400E4B10B574
:109A58000124C3F80445BFF36F8FBFF34F8F01EBA9
:109A68008204401AA14208D1074B0022C3F80425FA
:109A7800BFF36F8FBFF34F8F10BD431851F8042BFE
:109A88001A60FFF7ADFFEDE700E0014028B139B1FA
:109A98000023C1E900301846704748F2105070475B
:109AA80048F21350704738B1006848F24053884272
:109AB80014BF18460020704748F21050704730B164
:109AC80048F21153914214BF18460020704748F2DB
:109AD8001050704770B506460C461D46FFF7D6FF76
:109AE80050B9B3794AB1AB420AD111462046FFF7C3
:109AF8004DFA08B9044B236070BD48F21050FBE7DB
:109B080048F21150F8E700BF7052464D2DE9F04772
:109B18000C4606460F492046DDE9088915461F46CA
:109B2800FFF7C1FFA0B963685A7949465200404619
:109B3800FFF7C5FF60B94DB1CDF820803B462A46F6
:109B480021463046BDE8F047FFF728BA48F21050E2
:109B5800BDE8F0877052464D10B5044638B149B19A
:109B68000B684160984708B9044B236010BD48F260
:109B78000150FBE748F21050F8E700BF6E52464824
:109B8800F0B4134648B10768094EB7420AD161B12B
:109B98002AB14368F0BC5B68184748F2015318467D
:109BA800F0BC704748F20253F9E748F21053F6E761
:109BB8006E524648F0B460B107680C4EB7420CD1FB
:109BC80071B143681568DC68A5420CD3F0BC9B688A
:109BD800184748F20150F0BC704748F20250FAE7C3
:109BE80048F21350F7E748F21450F4E76E5246482B
:109BF800F7B50446DDE9086715460193FFF7ACFFA2
:109C080068B9019A29462046FFF7BAFF38B93A469B
:109C18003146204603B0BDE8F040FFF7CBBF03B0A4
:109C2800F0BD0000F8B50A4F0A4C0B4DE41B0121AA
:109C3800E40829700026A64203D102232B700020D5
:109C4800F8BD57F8363098470028F9D10136F2E7C1
:109C580040D7070040D70700E05B002001390144E6
:109C6800814200D2704703780A7800F8012B01F886
:109C78000139F5E7013A02440139824200D27047BE
:109C880011F8013F02F80139F7E770B516460D469D
:109C9800FFF7F0FF3246A9193044BDE87040FFF7DE
:109CA800E9BF38B50D460446FFF7D8FF29466019C5
:109CB800BDE83840FFF7D2BFBFF34F8F0549064BC9
:109CC800CA6802F4E0621343CB60BFF34F8F00BF52
:109CD800FDE700BF00ED00E00400FA0508B507281D
:109CE8001BD8DFE800F004121A1A1A041A0401201B
:109CF800FFF757FE0020FFF72DFE0120FFF72AFE91
:109D0800BDE808400220FFF731BE0120FFF72EFE14
:109D1800BDE808400220FFF71DBE08BD08B5FFF7E3
:109D2800CBFF08B5FFF7C8FF08B501F097FB4FF464
:109D38008051002001F02FF908B1FFF7BDFF054859
:109D4800C0F5FC2101F027F90028F6D1024801F0FE
:109D580047F8F2E700800700E59C07001AB1013ACE
:109D68008B5C8354FAE77047C3F10803DB0070B5D6
:109D780001330446002003A55B1920C940CAAD1968
:109D880020C4184720C940CA754120C420C940CA08
:109D9800754120C420C940CA754120C420C940CAA1
:109DA800754120C420C940CA754120C420C940CA91
:109DB800754120C420C940CA754120C4404170BDC6
:109DC8000000000000000000C3F10803DB0070B5CC
:109DD8000133002403A500BF5B1920C940CAAD1B8D
:109DE80020C0184720C940CAB54120C020C940CA70
:109DF800B54120C020C940CAB54120C020C940CAC9
:109E0800B54120C020C940CAB54120C020C940CAB8
:109E1800B54120C020C940CAB54120C06441B4FA48
:109E280084F0400970BD00BF2DE9F04F08B4F8CAAE
:109E380004B451F8042BA3FB028940F8048B4FF0BB
:109E4800000AE4FB629A4FF0000BE5FB62AB4FF0AF
:109E5800000CE6FB62BC4FF0000EE7FB62CE51F847
:109E6800042B4FF00008E3FB628940F8048BE4FB05
:109E7800629AE5FB62ABE6FB62BCE7FB62CE51F897
:109E8800042B4FF00008E3FB628940F8048BE4FBE5
:109E9800629AE5FB62ABE6FB62BCE7FB62CE51F877
:109EA800042B4FF00008E3FB628940F8048BE4FBC5
:109EB800629AE5FB62ABE6FB62BCE7FB62CE51F857
:109EC800042B4FF00008E3FB628940F8048BE4FBA5
:109ED800629AE5FB62ABE6FB62BCE7FB62CE40F848
:109EE800049B40F804AB40F804BB40F804CB40F8AE
:109EF80004EB0CBC052B00F01E810C68A0F11400CB
:109F0800A1F11401A2F1140252F804EB4FF000057C
:109F180050F8046BE4FB6E5652F804EB50F8047BDF
:109F2800E4FB6E6752F804EB50F8048BE4FB6E78A0
:109F380052F804EB50F8049BE4FB6E8952F804EBEA
:109F480050F804ABE4FB6E9AA0F1140052F8044BED
:109F580051F804EB4FF0000CE4FB6EC540F804CB5D
:109F680051F804EBE4FB6E5640F8045B51F804EB3F
:109F7800E4FB6E6740F8046B51F804EBE4FB6E7881
:109F880040F8047B51F804EBE4FB6E8940F8048B3D
:109F980051F804EBE4FB6E9AA0E80006062B00F0EB
:109FA800CA800C68A0F11800A1F11801A2F11802EA
:109FB80052F804EB4FF0000550F8046BE4FB6E56C2
:109FC80052F804EB50F8047BE4FB6E6752F804EB9C
:109FD80050F8048BE4FB6E7852F804EB50F8049BBD
:109FE800E4FB6E8952F804EB50F804ABE4FB6E9A7C
:109FF80052F804EB50F804BBE4FB6EABA0F1180078
:10A0080052F8044B51F804EB4FF0000CE4FB6EC51A
:10A0180040F804CB51F804EBE4FB6E5640F8045BBF
:10A0280051F804EBE4FB6E6740F8046B51F804EB5D
:10A03800E4FB6E7840F8047B51F804EBE4FB6E898E
:10A0480040F8048B51F804EBE4FB6E9A40F8049B4B
:10A0580051F804EBE4FB6EABA0E8000C072B6AD0C8
:10A0680008B40C68A0F11C00A1F11C01A2F11C02AB
:10A0780052F804EB4FF0000550F8046BE4FB6E5601
:10A0880052F804EB50F8047BE4FB6E6752F804EBDB
:10A0980050F8048BE4FB6E7852F804EB50F8049BFC
:10A0A800E4FB6E8952F804EB50F804ABE4FB6E9ABB
:10A0B80052F804EB50F804BBE4FB6EAB52F804EB27
:10A0C80050F804CBE4FB6EBCA0F11C0052F8044B22
:10A0D80051F804EB4FF00003E4FB6E3540F8043B05
:10A0E80051F804EBE4FB6E5640F8045B51F804EBBE
:10A0F800E4FB6E6740F8046B51F804EBE4FB6E7800
:10A1080040F8047B51F804EBE4FB6E8940F8048BBB
:10A1180051F804EBE4FB6E9A40F8049B51F804EB09
:10A12800E4FB6EAB40F804AB51F804EBE4FB6EBC07
:10A13800A0E8001808BCBDE8F08F10B5002253B2A3
:10A148008B4205DA1BB2002440F823400132F6E7BF
:10A1580010BD10B500231A465CB28C4204DA50F8E0
:10A16800244001332243F7E7B2FA82F0400910BDD8
:10A178004A11012301F01F0150F822008B401840BA
:10A1880070470139C9B24BB2002B0BDA013111F01B
:10A19800FF0315D059B201F18043013B50F8232049
:10A1A800002304E050F82330002BEAD0EEE712B188
:10A1B80052080133FBE7481E03EB401080B200E071
:10A1C800184600B2704730B5002463B2934206DAED
:10A1D8001BB2013451F8235040F82350F5E730BD45
:10A1E80010B5013AD2B253B2002B09DB1BB250F8BA
:10A1F800234051F823309C4204D8F2D2FF2002E0D9
:10A20800002000E0012040B210BD00EB81010023D6
:10A21800884206D251F8042D43EA52030B60D30753
:10A22800F6E7704770B59DF910401D46234606466F
:10A23800FFF79AFD30B9284631462246FFF7D0FF8E
:10A24800012807D0304631462A462346BDE87040EB
:10A25800FFF7BABD70BD70B59DF910401D46234685
:10A268000646FFF7B1FD38B1304631462A46234647
:10A27800BDE87040FFF778BD70BD00002DE9F043E0
:10A28800B3B002AC9DF9E8901F4680464B46204685
:10A29800FFF7CAFD22AB494638468DE81800FFF79C
:10A2A80070FFC0EB891086B2474B32B21340002BC7
:10A2B800BCBF03F1FF3363F01F034FF0200592FB8F
:10A2C800F5F5EDB2B8BF01336DB29CB212A82946BC
:10A2D800FFF733FF23B2002B28B213DD12AA0021A7
:10A2E80002EB80000A464A4513D257F8225005FA75
:10A2F80003F4214340F82210C3F1200125FA01F1AB
:10A308000132F0E712AB03EB800039464A46FFF70B
:10A318005AFF0FFA89F512AB6F00012403EB85058C
:10A32800330444D40022114653B2BB4222DA0DF161
:10A33800C80E0EEB840E0DF1C80C18B25EF8C8EC0E
:10A348000CEB83035EF820E053F8803CC3EB0E036C
:10A358005B1A734502D08CBF01210021C4F1010EA4
:10A368000DF1C80C0CEB8E0E01325EF8C8EC4EF8FD
:10A378002030D9E7621A544212A849465441FFF7DF
:10A3880044FF32AA09F1FF3302EB830302EB89028F
:10A39800284652F8801C53F8802C013E42EAC172CC
:10A3A800494643F8802CB6B2FFF72FFFB8E732AB27
:10A3B80003EB8404404654F8C81C4A46FFF703FFE1
:10A3C80033B0BDE8F08300BF1F00008030B51C46E5
:10A3D80091B0054693F900306846FFF725FDD4F89B
:10A3E800AC3028466946984711B030BD13460A4636
:10A3F800FFF7ECBF2DE9F04115468AB004468846C0
:10A4080002A80021202203F033F92E7803232046E6
:10A4180041462A462F1D76B20293FFF7E7FF2046F2
:10A42800214602AA3B460096FFF715FF2046214623
:10A4380042462B46FFF7CAFF00962046214605F103
:10A4480084023B46FFF7EEFE0AB0BDE8F08100004B
:10A45800F0B50C4689B008220646FFF7B4FEE36A59
:10A468000393236B0493636B0593A36B0693E36BCE
:10A478000793002769466A460823684602970197AA
:10A488000097FFF771FC314605466A4608233046B7
:10A49800FFF76AFC236B0393636B0493A36B059329
:10A4A800E36B0693054469466A460823684607979E
:10A4B800FFF75AFC314605446A4608233046FFF741
:10A4C80053FC236A0093636A0193A36A0293A36B04
:10A4D8000693E36B0793054431466A4608233046E2
:10A4E800059704970397FFF73FFC636A0093A36AF5
:10A4F8000193E36AA26B0293636B0393049206933E
:10A50800E26B236A05920544079331466A4608239D
:10A518003046FFF729FCE36A0093236B0193636BD2
:10A528000293236A0693A36A0793054431466A4651
:10A5380008233046059704970397FFF745FC236BDC
:10A548000093636B0193A36B0293E36B0393636ABA
:10A558000693E36A07932D1A31466A460823304664
:10A5680005970497FFF730FC636B0093A36B019387
:10A57800E36B0293236A0393636A0493A36A0593C4
:10A58800236B07932D1A31466A46082330460697EF
:10A59800FFF71AFCA36B0093E36B0193636A0393C1
:10A5A800A36A0493E36A0593636B07932D1A3146F4
:10A5B80030466A46082302970697FFF705FC2D1ACE
:10A5C80016D5304631460D4A0823FFF7CDFB45190D
:10A5D800F7D410E0094831460822FFF701FE0128A8
:10A5E80009D030463146054A0823FFF7EDFB2D1AFE
:10A5F800002DEFD0F5E709B0F0BD00BF7CD907000A
:10A60800F0B589B01C4607460E4615466846114601
:10A618001A46FFF7EBFE384639466A462346FFF7E7
:10A62800D5FE684669462A462346FFF7CFFE3046E0
:10A6380031466A462346FFF7C9FE09B0F0BD2DE949
:10A64800F0438BB08046129D15F9046B00961446B2
:10A658001F4689462B4602A811464246FFF7FBFDD6
:10A6680002A80146129AFFF7C1FE4046414602AAD7
:10A67800129BFFF7ABFE2046214602AA129BFFF76A
:10A68800A5FE2B46384639464A460096FFF7E3FDB5
:10A6980002A83946129AFFF7A9FE02A801464246C7
:10A6A8002B460096FFF7D7FD02A8014622462B4607
:10A6B8000096FFF7D0FD2046214642462B460096DD
:10A6C800FFF7C9FD484649462246129BFFF77EFE22
:10A6D8002046414602AA2B460096FFF7BCFD3846A5
:10A6E80039462246129BFFF771FE384639464A46DC
:10A6F8002B460096FFF7AFFD204602A93246FFF72A
:10A7080062FD0BB0BDE8F0832DE9F0478846B3F948
:10A7180002101F460825CB1D202493FBF5F51F3199
:10A72800954291FBF4F44FFA84F928BF1546064682
:10A738004946FFF702FD2A4630464146FFF70EFB21
:10A74800B7F90230ED009D4220D9ED1A06EB8401DD
:10A7580000228E420AD251F8040D20FA05F3134361
:10A768000B60C5F1200300FA03F2F2E724373846FC
:10A7780031464A46FFF734FD012807D030463146B6
:10A788003A464B46BDE8F047FFF71EBBBDE8F087E9
:10A79800F8B5036813F0010506460F46144605D0C0
:10A7A80001463A462346FFF7DFFA0546304621467A
:10A7B800FFF72BFD45B104F18042013A56F82230EB
:10A7C80043F0004346F82230F8BDF0B50646A1B084
:10A7D8000F460846194615461C46FFF7BAFC20B135
:10A7E80030462146FFF7A9FC73E068463946224601
:10A7F800FFF7E9FC08A829462246FFF7E4FC10A861
:10A808002146FFF79AFC012318A821461093FFF769
:10A8180094FC684608A92246FFF7E2FC002853D0BA
:10A82800009BDA0704D468462146FFF7EEFC26E0D1
:10A83800089BDB0704D408A82146FFF7E6FC3DE0A7
:10A8480000281EDD08AA234669466846FFF7BCFAB9
:10A8580068462146FFF7D9FC10A818A92246FFF739
:10A86800BFFC002805DA10A801462A462346FFF750
:10A878007BFA10A8014618AA2346FFF7A5FA10A8E4
:10A888001DE008A86A4623460146FFF79DFA08A876
:10A898002146FFF7BAFC18A810A92246FFF7A0FC2A
:10A8A800002805DA18A801462A462346FFF75CFA6D
:10A8B80018A8014610AA2346FFF786FA18A82946C1
:10A8C8002246FFF765FFA4E7304610A92246FFF7A6
:10A8D8007AFC21B0F0BD2DE9F04793F9006092B001
:10A8E800044689461046314615469846FFF731FC1E
:10A8F800002840F0978002A849464246FFF776FDB7
:10A9080043460AA8214602AAFFF760FD02A80146AD
:10A918004246FFF76BFD4346484649462A46FFF73D
:10A9280055FD08F10407284629464246FFF75EFD13
:10A93800204621462A463B460096FFF773FC2846E8
:10A9480029462A463B460096FFF76CFC28462146D6
:10A958002A463B460096FFF77EFC204621462A46BB
:10A968004346FFF733FD2846214622463B460096DC
:10A97800FFF758FC20463B46009621462A46FFF73B
:10A9880051FC2368DB07204613D5334621463A4657
:10A99800FFF7EAF9314682462046FFF736FC06F112
:10A9A8008043013B54F8230040EACA7044F823006E
:10A9B80002E03146FFF729FC284621464246FFF7C8
:10A9C80015FD284629460AAA3B460096FFF743FC90
:10A9D800284629460AAA3B460096FFF73CFC0AA8E7
:10A9E80001462A463B460096FFF735FC204621469D
:10A9F8000AAA4346FFF7EAFC02A802463B4621465C
:10AA08000096FFF728FC204629463246FFF7DBFB75
:10AA1800284649463246FFF7D6FB484602A9324641
:10AA2800FFF7D1FB12B0BDE8F0870000004870477F
:10AA380078D907002DE9F04FEFB01E46789D0590B4
:10AA48002B780393B5F9023092461F33202293FBEB
:10AA5800F2F3DBB206939DF9187095F9012007F11E
:10AA6800FF3926AB002443F829406EAB03EB89037A
:10AA78004EA88B46314643F8804C43F8604CFFF7AC
:10AA88006DF995F9012056A8B118FFF767F99DF9F6
:10AA98000C604EA83146FFF75CFB8046002840F06A
:10AAA800468156A83146FFF754FB0446002840F07B
:10AAB8003C8105F1240840464EA93A46FFF790FB31
:10AAC800012840F03481404656A93A46FFF788FBF2
:10AAD8000128089040F02B813B461EA856A9424603
:10AAE800FFF773FE0DF1380C6046594652462B4667
:10AAF8004CF82940CDF810C0FFF706FEDDF810C06D
:10AB08000097604661461EAA4346CDF824C00DF55D
:10AB1800BC79FFF7B3FB4346009716A84EA91EAAB7
:10AB2800FFF7ACFB484632460599FFF74CFBB300EC
:10AB3800049309EB030B049A059B5846991832466F
:10AB4800FFF741FB05F144031946324636A807933F
:10AB5800FFF739FB05EB860132463EA8443105F183
:10AB6800040AFFF730FB494600961EA836AA53464A
:10AB7800FFF771FB4A465B4636A83EA90095FFF7EA
:10AB88005EFD1EA8014633465246FFF71EFE1EAA6A
:10AB9800484659462B46FFF733FDDDF824C0079B8E
:10ABA8000B936046059B0C933946CDF814C00A9464
:10ABB800CDF83490FFF7E5FA3946044616A8FFF7B2
:10ABC800E0FAA042B8BF204684B2DDF814C0671E80
:10ABD8003FB260463946FFF7CBFA394610F1000913
:10ABE80016A818BF4FF00109FFF7C2FA002814BFD2
:10ABF8000223002343EA09090DF1280B32465BF8CA
:10AC0800297026A83946FFF7DEFA049B3246F91860
:10AC18002EA8FFF7D8FA31461EA8FFF78EFA023C95
:10AC2800089B1E93A6B20FFA86F9B9F1000F26AF5A
:10AC380047DB2B461EAAD5F8A44038462EA9A047C4
:10AC480049460EA8FFF794FA4946041C16A818BFEF
:10AC58000124FFF78DFA002814BF022300231C43A8
:10AC68000AAB53F82490B9F1000F27D09DF90C4096
:10AC780036A849462246FFF7A6FA049B3EA809EBE8
:10AC880003012246FFF79FFA36A83EA91EAA2B46C3
:10AC9800FFF7B6FC46A8394636AA53460094FFF794
:10ACA800DAFA36A83EA93A462EAB0095FFF7C7FC5C
:10ACB8001EA8014646AA2B46FFF788FB013EB6B2FE
:10ACC800B1E71EA8014652469DF90C30FFF77DFDFD
:10ACD80038462EA91EAA2B46FFF792FC9DF918406C
:10ACE800404639462246FFF77BFA012805D0384608
:10ACF800394642462346FFF767F8039B013BDBB220
:10AD080000245AB2002A0CDB12B26EA901EB8201B0
:10AD180057F8222051F8801C013B4A401443DBB20B
:10AD2800EFE7B4FA84F0400902E0404600E020462C
:10AD38006FB0BDE8F08F007800F00100704741DF88
:10AD480070470000014B01221A7070470460002010
:10AD5800BFF34F8F0549064BCA6802F4E0621343FC
:10AD6800CB60BFF34F8F00BFFDE700BF00ED00E0F1
:10AD78000400FA05024B034800221A7001F066BC71
:10AD88000460002059AD0700042810B5044609D80E
:10AD9800022811D816D00D4B1B68B3B12046BDE868
:10ADA80010401847831F012BF5D8094B094800228A
:10ADB8001A7001F04BFCEEE707494FF4701000F0F1
:10ADC8001BFAE8E701F08AFBE5E710BD0860002000
:10ADD8000460002059AD07007DAD070000207047D2
:10ADE80038B5554B554A18604FF0A0430020C3F8BA
:10ADF800402701F041FC0446002840F0988000F00C
:10AE0800D7FA012800F08E80022800F092800028EE
:10AE180040F08D804FF08043D3F8004414F4803420
:10AE280035D04FF48032C3F800240446444D2B6AD1
:10AE3800012B3FD04FF4701400F050FB414A202101
:10AE48001820FDF7B5FA08B1FEF76BFF3E4B1A68FC
:10AE580002F0F802B02A06D11A68D20742BF1A686F
:10AE680002F04E021A60FFF7B9FF00285FD12046B2
:10AE7800364900F0C1F9364800F0E6FC002856D102
:10AE880000F052FBFDF71EFBFFF759FFF8E7D3F878
:10AE9800202502F0F802A82A0AD1D3F82025D007E5
:10AEA80006D5D3F8202502F05602C3F82025BDE7C1
:10AEB8000124BBE743F204031A68264B9A4209D0DF
:10AEC80001F08AFCAA69014694B1234801F060FFA9
:10AED80090B9AFE76A6B1CB995F86032012BEFD0D7
:10AEE8001E484FF4805101F053FF0028E8D1A1E734
:10AEF80095F8A132012BE8D14FF0A043D3F81035D3
:10AF0800D90397D5104B1B6813F0B10F92D101F0FC
:10AF18000FFC60B9124B1870124801F097FB00F053
:10AF280025F804E00E4B10481C7001F08FFB03203D
:10AF380038BD4FF4A0247FE7086000200C00030010
:10AF4800D4770020E45B00201C0500407DAD07009D
:10AF580091AD0700DBE5B151757A0020347A002005
:10AF6800046000204DAD070059AD070008B5074B38
:10AF78004FF0FF32C3F88020C3F8802101F0D2F8E7
:10AF8800BDE808404FF4805000F032B800E100E01E
:10AF980080F30888084770B5C1F30B0434BBB0F5DB
:10AFA800FE2F23D84B1E1B0B020B03EB103101267F
:10AFB8004FF08040914201D2204670BD02F01F033D
:10AFC800550906FA03F3032D05D8DFE805F0020654
:10AFD800090CC0F800360132ECE7C0F80436FAE78D
:10AFE800C0F81036F7E7C0F81436F4E70724E3E7AB
:10AFF80010B504461448C0F5FE21FFF7CCFF08B190
:10B00800FEF78FFE01F0E8FB104B9B6903F6FF7318
:10B0180023F47F6323F00F0319180020FFF7BBFF09
:10B0280008B1FEF77EFEEFF305830023D4E90001A3
:10B0380083F3148883F3108883F3118883F31388C8
:10B04800BDE81040FFF7A4BF00800700D4770020B8
:10B0580037B56FF07F42154C057BD4F804358A422A
:10B0680028BF0A46891A13444A1E942A23F07F43AC
:10B0780005F5A8729BBF963B96314160416044F844
:10B0880022300B4B4FF4F86043F001039847094B0B
:10B09800AA00134400221A601B680193019B4FF415
:10B0A8008033AB40C4F8043303B030BD00400240E5
:10B0B80030DA07004041024018490A7884B0002A73
:10B0C80029D14FF08043A020D3F81834DB035EBFAA
:10B0D800134B01221A60134A00231360126803926B
:10B0E800039A114A136012680292029A0F4A136077
:10B0F80012680192019A0E4A82F8240310205060C7
:10B108000C4A0D48C2F80835012303600220136079
:10B11800C2F804030B7004B0704700BF1060002031
:10B1280008000040004102404041024044410240C2
:10B1380000E100E00040024008400240284B1A6845
:10B1480013B542B127490A6801320A6000221A6021
:10B158001B680093009B244B1A68A2B100221A6056
:10B1680022481B68027B0193019B4FF48033934074
:10B178001F4AC2F808334168044601BB8168D9B93F
:10B18800236803B198471B4B1A6832B300221A6030
:10B1980016481B68027F0193019B4FF4803393404C
:10B1A800134AC2F808334169044659B1103002B055
:10B1B800BDE81040FFF74CBFFFF74AFFE0E7FFF795
:10B1C80047FFE0E7816911B11030FFF741FF2369BC
:10B1D8001BB102B0BDE81040184702B010BD00BF57
:10B1E800044102400C600020404102407C5900208C
:10B1F800004002404441024070B50B4B1D682A7B59
:10B208004FF480339340094A0E46C2F80833044687
:10B2180040B1FFF751FF2E6021462846BDE8704037
:10B22800FFF716BF70BD00BF9C59002000400240C8
:10B2380070B5074B1D6804460E46A860FFF73CFF33
:10B248002E6021462846BDE87040FFF701BF00BFC9
:10B25800A0590020014B01221A707047116000208C
:10B2680070B5154DEA6A6E6AAC6CAC2A13D16B6B7B
:10B278001C44F61AEB6AAC2B13D010483246214610
:10B2880002F09AF9A8B100F04FF931462046BDE81E
:10B29800704000F029BF002CECD101F0B3FA04464D
:10B2A800E8E706483246A4F5804102F085F900280F
:10B2B800E3D1002070BD00BFD477002000800700D4
:10B2C8002DE9F74F06468846A8EB06052D0B02F632
:10B2D800FF77144600F002F9082D28BF08252B0334
:10B2E800DFF868B001933F0B0CB9234629E0BD4253
:10B2F8002CBFBA46AA464FF000025146304634BF2A
:10B30800DDF80490A14600F0D7FE0346C8B909F15C
:10B31800030222F003024146304600F0BFFE034616
:10B3280078B9DBF830304B44CBF8303001F094F981
:10B33800A7EB0A07A4EB09044E44C84403460028B7
:10B34800D2D0184603B0BDE8F08F00BFD4770020F4
:10B3580010B501F067FA154A42F20403916CCC5813
:10B3680003F1A34303F5471303F2D7539C4218D1C3
:10B37800D2E90C32934216D0884204D1BDE810407D
:10B38800002001F069B9D21A02F6FF7222F47F6236
:10B3980022F00F0219441844FFF792FF0028EDD05D
:10B3A80010BD0320FCE70020FAE700BFD477002097
:10B3B80070B5264CE36AAA2B37D005D8012B0BD0E1
:10B3C800A52B2ED0002070BDAC2BFBD1FFF7C0FF02
:10B3D80048BBFFF745FF26E0A66C656A01F0FCF95B
:10B3E800864229D101F0F8F900222946FDF7D4F860
:10B3F800A36A984202BF0123C4E90703A561002597
:10B40800134801F0DDF9134B134800221A7001F0BC
:10B4180023F968B975B1236A012B14BF01200220F2
:10B42800D1E7FFF795FF0125EAE7FFF719FFE6E700
:10B438000320C8E70120C6E7236BEA1AF11818446D
:10B44800FFF73EFF0028DAD1CCE700BFD477002011
:10B45800F8770020116000205DB2070040F6F87010
:10B4680008B50368013302D10749FEF7D9FA40F657
:10B47800FC700368013305D1BDE808404FF4FC2196
:10B48800FEF7CEBA08BD00BF008007000A4AD2F80E
:10B4980000347BB109480023D2F80815D940C90700
:10B4A80048BF03F5C07103F1010348BF42F821000A
:10B4B800072BF1D1704700BF000001403546526E9E
:10B4C800FFF7E4BF044B002282B01A601B680193A7
:10B4D800019B02B0704700BF0001014038B50E4C17
:10B4E8002278BAB90D4BD3F800248AB1D3F80455A1
:10B4F800FFF7CCFF40F61650A842B8BF28460849C7
:10B50800A0F54860FFF794FE064B4FF480321A60AE
:10B518000123237038BD00BF1260002000000140E5
:10B52800C9B4070000E100E0034BD3F800340BB1C5
:10B53800FFF7ACBF704700BF00000140044B18681C
:10B54800421C04BF034B1878831F58425841704768
:10B5580030010010E00F00F0074B1B78062B09D1D3
:10B56800064B1B68C3F30313033B032B02D8044A9F
:10B57800D05C704700207047E00F00F0E80F00F043
:10B588003EDA070008B5FFF7D9FF28B1834B844A94
:10B598001B68C3F304231360FFF7DEFF10B1814B70
:10B5A800814A1A60FFF7CAFF28B1804B804A1B689E
:10B5B800C3F342331360FFF7CFFF20B17D4AD3684E
:10B5C80023F08073D360FFF7B9FF40B14FF0804399
:10B5D8000022C3F80C21C3F81021C3F83825FFF75F
:10B5E800BBFF10B1744B03221A60FFF7B5FF40B1DF
:10B5F800724B05221A6001229A6700229A603F2244
:10B608005A606F4B1A68511C0BBF6E4B6E4B1A7801
:10B618001B6802BF08331B68C3F30313062A4DD106
:10B62800033B032B03D8694AD35C002B46D04FF069
:10B638008052674BD2F80414C3F82015D2F80814C6
:10B64800C3F82415D2F80C14C3F82815D2F810142E
:10B65800C3F82C15D2F81414C3F83015D2F81814FE
:10B66800C3F83415D2F81C14C3F84015D2F82014C6
:10B67800C3F84415D2F82414C3F84815D2F828148E
:10B68800C3F84C15D2F82C14C3F85015D2F830145E
:10B69800C3F85415D2F83414C3F86015D2F8381426
:10B6A800C3F86415D2F83C14C3F86815D2F84014EE
:10B6B800C3F86C15D2F84424C3F87025FFF73EFF91
:10B6C80028B1444B444A1B6803F04F031360FFF74B
:10B6D80035FF48B14FF08043D3F80024D20744BF68
:10B6E8006FF00102C3F80024354B1B68062B0CD100
:10B6F800354B1B68033B032B02D8384AD35C23B174
:10B70800374A136843F480631360364AD2F88830A6
:10B7180043F47003C2F88830BFF34F8FBFF36F8FC5
:10B728004FF01023D3F80022002A03DBD3F80432A9
:10B73800002B2FDA2C4B0122C3F80425D3F8002460
:10B74800002AFBD04FF010221521C2F80012D3F8BE
:10B758000024002AFBD04FF010231522C3F804223E
:10B76800214B1A46D3F800140029FBD00021C3F856
:10B778000415D2F80034002BFBD0BFF34F8F1949C2
:10B788001A4BCA6802F4E0621343CB60BFF34F8FD1
:10B7980000BFFDE7164B174A1A6008BD24030010C6
:10B7A8004035014074C007400DF0ADBA44020010A6
:10B7B8003C050040F0ED00E0A005004010560040B8
:10B7C80030010010E00F00F03401001036DA0700F5
:10B7D80000C0004058020010E40E00403ADA0700AA
:10B7E8003C17004000ED00E000E001400400FA05CD
:10B7F800A45900200090D00313681F2B10B51446DD
:10B8080007D900220830FDF740FB08B92023236040
:10B8180010BD48F21450FBE70830FDF713BB0830A1
:10B82800FDF7E0BA831F012B10B5044602D80020AB
:10B8380000F0AEFF034B1B681BB12046BDE810406B
:10B84800184710BD1460002008B5074B1860002089
:10B85800FFF7E8FF054800F083FF20B9BDE808407E
:10B86800024800F0EFBD08BD146000202DB80700A5
:10B878006CDF70476DDF704772DF704773DF7047AA
:10B8880074DF704775DF704776DF70477ADF70477F
:10B898007CDF70477DDF70477FDF704786DF70474A
:10B8A8008FDF704790DF7047A8DF7047AADF7047C7
:10B8B800ADDF7047AEDF7047B0DF7047B1DF70476C
:10B8C800B5DF704762DF704766DF704713DF704788
:10B8D8007FB50023CDF80B308DF80F300A4BADF84B
:10B8E80006109B89ADF8083001238DF80A300DF158
:10B8F8000603CDE90430054B02A91888FFF7DAFFE3
:10B9080007B05DF804FB00BF82700020AA59002030
:10B9180001460148FCF75FBF54D7070070B51822ED
:10B928008CB000210DEB020001F0A2FE2823089341
:10B9380016231E4CADF806300023CDE903330593DA
:10B948000223092606222370237159230125A27098
:10B9580063710322FE230DF10601A0198DF818501A
:10B968008DF82D500294ADF80C606570E270A371EB
:10B97800FFF790FFB8B9BDF8063026725A19E27180
:10B98800BDF80C200A4C134402A906AA2046ADF8BB
:10B998000C30FFF771FF30B92078FFF771FF20787E
:10B9A8002946FFF76BFF0CB070BD00BF96700020F2
:10B9B800A85900202DE9F0410388232B8AB00446BA
:10B9C80036D80F2B05D8012B00F0F2800AB0BDE85D
:10B9D800F081103B132BF9D801A252F823F000BFD5
:10B9E80069BA070085BA0700D5B9070055BB070033
:10B9F800B5BC0700D5B90700D5B90700D5B9070008
:10BA0800D5B90700D5B90700C3BC0700D5B90700E9
:10BA1800D5B90700D5B90700D5B9070087BB070016
:10BA2800D5B9070095BB0700D5B9070045BB070086
:10BA3800503B9AB2062AC9D8062BC7D801A252F899
:10BA480023F000BFADBA0700C5BB0700C3BC0700A1
:10BA5800D5B90700D5B9070005BB0700A5BB070086
:10BA6800994B82881A80994A12681C460AB10120AB
:10BA7800904797492088FFF705FFA7E7924B4FF6B5
:10BA8800FF721A80934B1B685A0704D4FFF746FFCE
:10BA980008B1FEF746F98D4B1B68002B96D00220A3
:10BAA800984793E78C4EE288B3889A428ED18B48A8
:10BAB800FCF76DFE0546002888D0228A04F11201A1
:10BAC80001F0ADFD1822002104A801F0D1FD0823E2
:10BAD8008DF81030824B0693824B0596CDE90735D9
:10BAE80004A8238AADF8243000F0A2FC00283FF413
:10BAF8006DAF7A482946FCF76EFE67E7E188F629BC
:10BB08001AD8CB1E9B070DD0CB1F9BB2013B5A42C4
:10BB180002F0030203F0030301F1FF3158BF53425F
:10BB2800C91A89B2684B1888FFF7CAFE00283FF483
:10BB38004DAFFEF7F6F849E7F721F3E7002204A92D
:10BB48008088CDE90422FFF7ADFEEFE700235E4CC5
:10BB5800ADF812300223ADF81030208802AB04AAE9
:10BB680042F605210593FFF7A3FE08B1FEF7D9F8C1
:10BB7800002320881A468521FFF78EFED6E7524B10
:10BB880000F108011888FFF77DFECFE7002304A91C
:10BB98008088ADF81030FFF783FEC7E7A379002B44
:10BBA8007FF414AF484B13211888FFF76DFEBDE7EB
:10BBB800454B00211888FFF787FEB7E7A379002BCC
:10BBC8003FF404AF022B7FF401AF434920898A89EF
:10BBD80090420E467FF4FAAEA27B012A7FF4F6AEBD
:10BBE80000220120CDE904228DF81600208A364D66
:10BBF800ADF81800608AADF81A0004F11400079037
:10BC0800ADF80A20098A28888DF8103001AF02AAF9
:10BC1800ADF808300397FFF74BFEA84660B93846E1
:10BC2800FFF789F840B940F2FD132888ADF81430C1
:10BC380004A9FFF741FEC9E6002304A9B8F80000EB
:10BC4800ADF81430FFF738FE014600287FF4BEAE89
:10BC5800182204A801F00CFD237D214A8DF810302C
:10BC6800022B0596069218D0062B10D0012B10D166
:10BC78001D4B1A881D4B1A80637DD4F81620089333
:10BC8800012B099205D11A4800F082FD01E0637D7D
:10BC9800089304A800F0CCFB98E6A27D637D43EAF4
:10BCA8000223114A1380114A1380F2E700231A462F
:10BCB80019468088FFF7F2FD38E70023A0881A4666
:10BCC8001946FFF7FBFD31E7AA590020BC70002098
:10BCD80036DC0700B87000208270002054D70700B7
:10BCE80069BD070019B90700C0700020C2700020A4
:10BCF80040D70700154938B50B68024613F0010014
:10BD080022D0134882421ED0124A10884FF6FF7282
:10BD1800904213D043F004030B601321FFF7B4FDE6
:10BD280090B90D4DC82445F001054FF47A40A84755
:10BD3800013CFAD1BDE8384001F012BB074B187836
:10BD4800FFF79EFDF6E7002038BD00BFB870002061
:10BD580040D70700AA59002030DC0700A859002066
:10BD680010B5044686B000210D2202A8019101F009
:10BD78007FFC2378082B0BD1364A3749138809886A
:10BD8800013B9BB21380D9B1D3B90323118023702F
:10BD9800627823788DF805306021012A8DF8041027
:10BDA8008DF806200ED00B2A12D100F093F98DF8E9
:10BDB8000700002000F088F9042101A8FFF788FD9A
:10BDC80006B010BD062B05D0082B29D0032B27D091
:10BDD8000321F2E7E1688DF80710D4E90123080A86
:10BDE8008DF80800080C090E8DF80A10110A8DF854
:10BDF8000B208DF80C10110C120E8DF80E201A0A5B
:10BE08008DF80F308DF810201A0C1B0E8DF80D10C0
:10BE18008DF809008DF811208DF812300F21CCE72C
:10BE2800D4E90123110A8DF807208DF80810110CA8
:10BE3800120E8DF80A201A0A8DF80B308DF80C2096
:10BE48001A0C1B0E8DF809108DF80D208DF80E3088
:10BE58000B21B2E7C2700020C07000202DE9F0432A
:10BE6800444B95B005464FF6FF721A8001204FF6F5
:10BE780059632A4602A98DF80A00ADF80830FFF781
:10BE880013FD0446002871D13B4B04AA03F11007A7
:10BE9800164618685968144603C40833BB4222463C
:10BEA800F7D1A91C3046FFF70DFD044600285DD1E7
:10BEB80001461C220DA801F0DBFB9DF83430ADF8DB
:10BEC800044043F004038DF834300223ADF80C30FD
:10BED800AB788DF80E3004F0F80343F003038DF8C7
:10BEE8000630F423CDE90A44ADF82C302B4601AED8
:10BEF80033F8040B0C944FF0110903AF08AA0DA9ED
:10BF0800CDE908768DF80590FFF7D0FCA0460446E9
:10BF180060BB01461C220DA801F0AAFB9DF8343035
:10BF2800ADF8044023F0180343F018038DF83430BB
:10BF38000123ADF80C30AB788DF80E301723CDE91E
:10BF48000A44ADF82C302B4608F0E80833F80C0BFF
:10BF58000C9448F0130808AA0DA9CDE908768DF8C5
:10BF680005908DF80680FFF7A1FC0446204615B021
:10BF7800BDE8F083AA59002018DC070030B5334C1F
:10BF8800236813F0010585B05DD1314B1860314845
:10BF9800FCF7E6FB029500F0B8F800284CD12E48D3
:10BFA800FFF794FC002847D101F09CF9002843D101
:10BFB80002A801F065FA00283ED102A9012001F08B
:10BFC80069FA002838D102A801F0CCFA002833D148
:10BFD80000F09EFB30B1214800F08EFB236843F04F
:10BFE80002032360112302A88DF80430FFF742FCF6
:10BFF80010BB9DF8093002A801338DF80930FFF70E
:10C0080037FCC8B923689B0718D5144988690431D7
:10C0180082B201A8FFF73CFC70B91148FFF736FC63
:10C0280050B91048FFF71AFF30B9FFF777FC18B975
:10C03800236843F00103236005B030BD0A4801F0CE
:10C048004AFB0949E4E70020F6E700BFB870002082
:10C05800BC70002054D7070000800700186000203B
:10C0680036DC07008270002010DC070043690BB142
:10C07800C06818477047000010B40549054C0022F5
:10C08800904218BF214604485DF8044BFCF7BDBB3D
:10C09800B8D70700E4D707006859002007B5009310
:10C0A80013460A4601460348FCF7B3FB03B05DF8A4
:10C0B80004FB00BF6859002013460A4601460148A0
:10C0C800FCF7AEBB68590020014B18700B20704775
:10C0D800C4700020024B002218781A70704700BF05
:10C0E800C470002018DF704730B585B005461022AF
:10C0F8000C466846002101F0BBFAA4086846019581
:10C108000294FFF7EFFF05B030BD1FB50023CDE95E
:10C1180001330393684602230093FFF7E3FF05B05A
:10C128005DF804FB4FF000534FF480521A60002072
:10C1380070470000014B06201B681847D07000208C
:10C148000A2803D90B38C0B2FFF7BEBF70470000FA
:10C1580010B5044686B00020FCF76AFB014630B1F2
:10C16800164A18212046FCF747F906B010BD1822D8
:10C17800684601F07DFA0423114A8DF80030114B0E
:10C18800116D1B68994211D10F4B186800F070FFB0
:10C198008DF80100FFF7D4FFD4E901138DF80100F1
:10C1A80068469847094800F057FADEE701238DF8FA
:10C1B80001306846D4E901139847D6E759C107000A
:10C1C800D4770020C8700020CC7000203DC1070043
:10C1D800F0B5044687B018220021684601F048FAF5
:10C1E80022788DF8002001238DF80130531E0B2B87
:10C1F80000F21281DFE813F01D0010001D001D0081
:10C2080010011D0010011D001001100110010C008B
:10C21800824B07201B689847D4E901136846984762
:10C228009DF80130012B00F0EC807C4B05201B6849
:10C23800E6E0062A7A4901D0012A01D122690A706A
:10C248000A78012A04D0022A53D000230B7093E005
:10C25800072BE1D801A252F823F000BF85C20700DE
:10C2680021C20700EFC20700C3C2070021C20700AE
:10C27800E9C2070021C207009DC20700674B0320DF
:10C288001B689847606900F0D1FCFFF759FF8DF8EB
:10C298000100C1E7A18A206900F0E0FCFFF750FF28
:10C2A800604B8DF80100DA6B1B6C0293E368019216
:10C2B800002BB1D020699847AEE75B495B4800F096
:10C2C8001BFDFFF73DFF01288DF80100A4D10020D8
:10C2D80000F0C2F900289FD00A238DF801309BE7AF
:10C2E8004FF4007303934F4BDA6B1B6C019202936C
:10C2F80092E7072B90D801A252F823F025C3070034
:10C3080021C20700DBC30700E5C3070021C20700FD
:10C318000FC4070021C2070085C3070000F0BEFC58
:10C3280008B90823D9E762690AB90323D5E7C2F334
:10C338000B0333B13B4B3C495B6D096813448B429B
:10C34800F3D1B2F5805F01D90423C6E7354B3649EE
:10C35800586D096815188D42E3D85A64DA6C9A64E6
:10C3680018651863314B1B68002201211844FFF738
:10C37800A3FE00283FF450AF0523AEE700F08EFC83
:10C388000028CED0274DA18AD5E914329B1A6A6CB1
:10C398000B449342C9D8254B2F6B1B68206905F1C4
:10C3A80048021F44FCF7F8F8E368A28A21690646A8
:10C3B8003846FFF773FE08B1E3687BE7A38A2A6B68
:10C3C800AE641A442A632A6D029613442B650193BE
:10C3D80022E7144B9A6C02921B6DF8E7114BD3E9D4
:10C3E8001402596C821A8A429BD19A6C58650021B2
:10C3F80020465964DA64FFF7ABFE084B1B6804203B
:10C40800984707B0F0BD074B9A6C1B6D01934FF42A
:10C41800805302920393FFE602235EE7D070002068
:10C42800AC590020D4770020C8700020CC700020C0
:10C4380083681BB1024A1821FBF7DEBF072070474B
:10C44800D9C1070038B50546C0B10120FFF714FE71
:10C45800044648B900F0DCFB00F020FC30B9084B7A
:10C4680000201D60FFF730FE204638BD054906480C
:10C4780000F042FC0128F2D00324F5E70724F3E793
:10C48800D0700020C8700020CC7000202DE9F04149
:10C4980015464FF46072064688461F4601F08CF830
:10C4A80028B915B90020BDE8F081A847FAE70022AD
:10C4B80001213046FFF700FE70B94FF46072414623
:10C4C800384601F0ACF82B464FF4607239463046D6
:10C4D800FFF7E4FD0028E5D00320E4E72DE9F0416B
:10C4E8003D4C236801335CD000225821201DFCF705
:10C4F80053F8D4F80080A8EB0002D2F1000848EB0A
:10C508000208364D364E2F683B6801335ED0002254
:10C518005821381DFCF740F83B68834244D17C68B9
:10C52800012C0AD00022C32107F51870FCF734F853
:10C53800D7F85C42231A5C425C41B8F1000F35D051
:10C54800254927484FF4607201F069F864B12968F9
:10C5580024485422043101F062F8296822484FF433
:10C5680032725C3101F05BF87468012C2CD11F49E0
:10C57800402201F5E47001F052F81D491C2201F532
:10C58800E47001F04CF81B4986F8A142002304220C
:10C5980001F2862086F8603286F8E23201F03FF830
:10C5A80010E04FF00008ACE70024C6E724B1296882
:10C5B8000B484FF46072D5E709484FF460720021C8
:10C5C80001F056F802237360BDE8F081B8F1000F5E
:10C5D800F2D00024B4E700BF00F00700B0590020F3
:10C5E800D4770020D87700203078002030790020D8
:10C5F80070790020F077002070B50C4C05460022B9
:10C608005821201DFBF7C8FF00222060C32104F534
:10C618001870FBF7C1FF2A46C4F85C022146044B98
:10C628000448BDE87040FFF731BF00BFD477002051
:10C63800D470002000F0070002460248024B006850
:10C64800FFF724BFB0590020547400200149FFF7B8
:10C65800F3BF00BF00F0070038B505460020FFF71C
:10C66800CBFF044618B903492846FFF7E5FF2046E3
:10C6780038BD00BFD477002010B5FFF7FDFC044695
:10C6880028B9FFF72BFF2046FFF7E6FF00B103208C
:10C6980010BD000010B5084C4FF40072FF2104F1E2
:10C6A8005C0000F0E5FF2022002104F1380000F0D2
:10C6B800DFFF0023236310BDD477002029DF7047F4
:10C6C80038B50C4D0446D5F8643378B101330FD131
:10C6D800002218210430FBF75FFF21462060072263
:10C6E80005F55970BDE83840FFF7E8BF0E2038BDA2
:10C6F8000820FCE700F0070008B528B103491C2210
:10C7080000F08DFF002008BD0E20FCE764F3070051
:10C7180010B5064C002218212046FBF73DFF54F8BF
:10C72800043C1B1A5842584110BD00BF68F307006B
:10C7380010B50A4CD4F82433D4F8642313400133D9
:10C7480009D04FF4FE20FDF753F9C92221464FF4D2
:10C75800FE20FDF77BF9002010BD00BFD477002034
:10C76800F8B5094E094CA41B0746E4080025A54264
:10C7780001D10020F8BD56F83530384698470028D2
:10C78800F8D10135F3E700BF40D7070048D70700C5
:10C79800F8B5094E094CA41B0746E40800250436E1
:10C7A800A54201D10020F8BD56F8353038469847E3
:10C7B8000028F8D10135F3E740D7070048D707002C
:10C7C80008B50C22002100F053FF024B00221A6327
:10C7D80008BD00BFD477002043F204031A68084B51
:10C7E8009A4201BF43F20803186800F6FF7020F46C
:10C7F8007F600CBF20F00F004FF48050704700BFDF
:10C80800DBE5B15108B5FFF7E7FF054B9B69184415
:10C8180000F6FF7020F47F6020F00F0008BD00BF15
:10C82800D47700204FF48050704700002DE9F74F6F
:10C838000193244BDFF894B01B6ADFF894900093BF
:10C84800054616464FF0000843F2040AB8F1010FF6
:10C858005FFA88F714D0022F1FD0FFF7D3FF6EB10D
:10C86800009B013B5C425C41A9EB0000A84200D35D
:10C87800F9B1B4B1A8421CD204201FE03446F3E752
:10C88800FFF7AAFF019B33B9DAF80040B4EB0B04B9
:10C8980018BF0124E8E74446E6E701244FF4805036
:10C8A800E2E708F10108B8F1030FCFD1A842E3D3BA
:10C8B80000E017B10448FFF783FF002003B0BDE88C
:10C8C800F08F00BFD4770020EC770020DBE5B15172
:10C8D8000050070090F8552012F0FB0F07D190F890
:10C8E800643023B1836ECBB10B600120704712F026
:10C8F800010303D090F8563003B1836D9207F2D547
:10C9080090F85C20002AEED0054A006EC2F5FC22A1
:10C91800904201D80344E6E7042070470F2070478F
:10C92800008007005B68DA680D4B9A4230B508D181
:10C938000C490A6812B90C4A14681CB10B4B002246
:10C948001A7030BDD0E90134181913F9015B002DB4
:10C95800A0EB0304F9DB0B601460044B0122EFE742
:10C96800ECDA07007C7B0020787B0020807B0020AD
:10C9780043F2040310B519491C688C4202462BD0B7
:10C9880042F20403C358581A434243418C421846A2
:10C9980021D142F20403D358A3421CD14FF440538F
:10C9A80002F500511B780978142B81BF43F2140358
:10C9B8000B481B68B3FBF0F398BF0023142989BF09
:10C9C80042F2140100205058054A88BFB0FBF2F02B
:10C9D800181A18BF012010BD0023D7E7DBE5B151B5
:10C9E80040420F002DE9FF472F49304D8A6B304CEC
:10C9F800304FDFF8D490DFF8D4A06E465C31304673
:10CA0800FCF77AFC96E80F0085E80F0000212A4B16
:10CA180039704FF447722046C9F80010CAF8001060
:10CA2800EB6000F025FE254922462846FCF7FFFE6C
:10CA380020B90027384604B0BDE8F0873F78002FBA
:10CA4800F7D094F86C3194F800801BB3B8F1000F5C
:10CA5800EFD194F87231002BEBD0DAF80020D9F836
:10CA680000103046FCF748FC96E80F0085E80F00F8
:10CA78004FF4B272414604F5BA7000F0F9FD10495E
:10CA880004F5BA722846FCF7D2FE0028D1D004F586
:10CA9800BA7406E0B8F1000FCBD0A379002BC8D048
:10CAA8000834084B1C60C5E7D4770020A07E00201E
:10CAB800847B0020807B00202DC90700A0DB0700B5
:10CAC800ECDA07005C7F00207C7B0020787B00206C
:10CAD80000B591B0FDF7A6F8684608492022FDF791
:10CAE800D4F86A46064907484023FCF7F3FF064B8B
:10CAF80001221A7011B05DF804FB00BF38D9070095
:10CB0800B07E002004D90700547B0020F0B5A3B004
:10CB180007460D4614461E4678222023002104A805
:10CB2800029300F0A5FD00230393194B1B780BB962
:10CB3800FFF7CEFF2DB337BB02AB164F0193164953
:10CB4800289B0097324604A8FDF752F8E8B9402C14
:10CB58001BD1124E22462946304600F060FD2021A6
:10CB68003046FDF79EF8CDE90064029B0C493A4631
:10CB780003A8FCF7CBFF00280CBF0120052023B039
:10CB8800F0BD1320FBE71620F9E70A20F7E700BFFE
:10CB9800547B0020F87E002044DA0700187F00202C
:10CBA800B07E0020F0B5ABB004460D4616461F46D1
:10CBB8007822202300210CA8039300F059FD114B83
:10CBC8001B780BB9FFF784FF2FB12146202204A858
:10CBD800FDF750F804AC03AB0B4F01930B490097DA
:10CBE80033462A460CA8FDF703F848B92022214607
:10CBF800384600F0E1FCB0FA80F040092BB0F0BDF7
:10CC08000020FBE7547B0020557B002044DA070016
:10CC180008B5044B986B08B1FFF7E4FE024B187097
:10CC280008BD00BFD4770020587F002010B5044607
:10CC380058B1B0F5007F0AD8064B00221A70FFF7EA
:10CC480029FD054B01209C6310BD0320FCE704204F
:10CC5800FAE700BF587F0020D477002070B50E4C4B
:10CC68000646E06BA36B42189A420D4611D85C3019
:10CC78000A462044314600F0D2FCE36B04F140023E
:10CC88002B4429463046E363FBF786FC20640120E9
:10CC980070BD0320FCE700BFD4770020014B187853
:10CCA800704700BF587F002013B5104C94F86C21D2
:10CCB800B2B194F8D802B4F8DA2204F5377104F561
:10CCC800B8740B4B1B6800930A4B1B68FFF71EFFD9
:10CCD800012809D1201D02B0BDE8104000F0CCB9F0
:10CCE800114610460434ECE702B010BD847B0020E6
:10CCF800787B00207C7B0020204BD3E90E329A42BF
:10CD08002DE9F04106460D4633D1DFF8788098F8D2
:10CD180000704FB1FFF776FD194B3060294618684F
:10CD2800BDE8F041FFF7D6BDFFF75CFE18B3FFF78B
:10CD3800BBFF0128376004462F6017D1104B2946E6
:10CD48001868FFF7C7FD012804460FD103463A4685
:10CD580028683946FFF76AFD38B9FFF753FD88F8A8
:10CD6800004030602046BDE8F0810424FFF792FCC3
:10CD7800F8E70824F6E70524F4E700BFD477002095
:10CD88005C7F0020587F002001237230FFF70ABF24
:10CD980013B50446084623781146032B03D8DFE869
:10CDA80003F021050F18002002B010BD0022D4F8AE
:10CDB8000140FBF7F1FB844214BF00200120F3E798
:10CDC8000A4600230146601C02B0BDE81040FFF788
:10CDD800E9BE009103464022611C0020FFF796FE41
:10CDE8000128E9E70120DFE72DE9F043A3B0044675
:10CDF8000D461746002178221E4604A820239DF8D8
:10CE0800AC900393DDF8A88000F032FC41220021A9
:10CE1800204600F02DFCB5F89430BB4282BF442375
:10CE280003FB075393F8969084F80090B9F1030F29
:10CE38001ED8DFE809F00902111F002241463046DA
:10CE4800FBF7AAFBC4F80100424631462046FFF72B
:10CE58009FFF23B0BDE8F08303AB0193631C0093ED
:10CE68000B494346324604A8FCF7C2FE0028EBD023
:10CE78000020EEE7442000FB07F2AB1802F19A010C
:10CE88002944B3F89820601C00F0C9FBDCE700BF18
:10CE980044DA07002DE9F0476F4B1D68A4B004463B
:10CEA8000F4690460A4601462846FFF76DFF0028C0
:10CEB80000F0D08095F8556026BB4FF00109CDE908
:10CEC800007923463246294613A8FFF78DFF00282C
:10CED80000F08380B8F1000F6ED041225F4813A99B
:10CEE80000F09DFB5E4B6A68C3F82C901E629A6046
:10CEF800002239462046FBF74FFB594B0125C3E971
:10CF08000970A2E04122002102A800F0B1FB06F05E
:10CF180001094122002113A806F0020600F0A8FB2F
:10CF2800B9F1000F4CD042F20403E15803F1A343D6
:10CF380003F5471303F2D75399424ED1D5F858A0B9
:10CF48000AF5FF530AF6FF72C2F30B021F339B1A4E
:10CF580042F20802A2589A423FD343F204031B68E4
:10CF68008B4213D14FF440531B78102B8ABF43F2E6
:10CF7800100300221A6804F500531B78102B8ABF8F
:10CF880042F210030023E3589A4226D12046FFF7C5
:10CF9800EFFC00B10EB30123CDE900A30022234624
:10CFA800294602A8FFF720FFB8B1AA6DA318BA1A3C
:10CFB8004EB9B8F1000F1AD1294B01255D6112E075
:10CFC8003A462346F4E70021CDE9002113A84A4652
:10CFD8002946FFF709FF0028EBD10525B8F1000F16
:10CFE80030D1FFF757FB284624B0BDE8F087DFF8BB
:10CFF8007080B9F1000F21D02046FFF7B9FC18B1B5
:10D0080008F11800FFF7DCFB1648412202A900F0DE
:10D0180006FB002E14BFAC23A523C8F82C30AB6D3B
:10D02800C8F83430002E3FF463AF0F48412213A9EB
:10D0380000F0F5FA6B68C8F80C3059E7AA23C8F86D
:10D048002C30EFE70948FFF7BBFBFFF723FB044B46
:10D058009C64C8E71725C1E75C7F0020757A00202B
:10D06800D4770020347A0020B67A0020F8770020A0
:10D078000122FFF70FBF000090F85420F0B50346D7
:10D08800002A51D090F8550003284DD893F86E2007
:10D09800032A47D11A7A002A46D0DA68342A45D1B9
:10D0A80043F204011A8A0C6821498C422AD152B1F0
:10D0B8005969E9B1D2B2002103F1140543F20C0613
:10D0C800CCB2A24201D8122011E055F82170348860
:10D0D800A74201F10101F3D11A78FAB101285B687E
:10D0E800144A15D89068834234BF10200120F0BD3F
:10D0F80010B9012AE7D8EFE7421E18BF0122002A1B
:10D10800EAD1E0E712B15A69002ADCD11A78F6E7C9
:10D11800D06883428CBF01201020E8E7012818BF9F
:10D128000F20E4E71420E2E70F20E0E71120DEE714
:10D13800DBE5B151D477002038B1054B0360054BCE
:10D14800436001230372002070470E20704700BF20
:10D1580087D1070061D1070069B10B78022B0CD188
:10D16800022804D0032814BF082011207047032385
:10D178000B70002070470E2070470820704710B5CC
:10D188000C4681B10B78012B06D00ED9033B012B3D
:10D1980094BF0820112010BDFFF792FA0028FAD199
:10D1A80002232370F7E70E20F5E70820F3E70000D5
:10D1B80070B5144B144A0C21D21AB2FBF1F28169F2
:10D1C80011F8025C044635B900690021914205D185
:10D1D800012323600EE04FF0FF30F6E71E68AE42F1
:10D1E8000CD1461C07D19D68D4E90001D4E902237B
:10D1F800A847206070BD5E688642F4D001310C33C8
:10D20800E4E700BF48D7070054D707001EF0040F13
:10D218000CBFEFF30880EFF30980FFF7C9BF00BF29
:10D2280010DF704711DF704713B504460949684697
:10D23800FBF724FD019808B902B010BDD0E9002120
:10D248002046904718B16846FBF722FDF2E7112007
:10D25800F2E700BF44DC070013B5044607496846F7
:10D26800FBF70CFD019B0BB902B010BD2046D3E9BA
:10D27800002190476846FBF70BFDF3E75CDC0700ED
:10D28800084B9A6822B11A6822F480021A60704723
:10D29800054B4FF48002C3F88020BFF34F8FBFF3D4
:10D2A8006F8F7047C859002000E100E00B4991F8E2
:10D2B80016335A09EC231341DB0706D5084B9A6845
:10D2C8003AB94FF480030B60704742F20200FCF752
:10D2D80028BD1A6842F480021A60704700E100E035
:10D2E800C8590020F7B5194F3C7864BB184E012582
:10D2F80020463570FFF798FF112821D02046FFF708
:10D30800ABFF144B8DF80340186801900DF1030032
:10D31800FBF708F9104901A8FFF782FF0446B0FAA5
:10D3280080F0400938709DF80300FBF71FF93CB9FD
:10D338000A4B34701C70FFF7B9FF2846FFF78CFFC3
:10D34800204603B0F0BD0824FAE700BF617F002043
:10D35800607F00203EDC0700259D0700627F0020DB
:10D36800F7B5154F3B781BB3144E01203070FFF70B
:10D378005BFF11284FF000051CD00220FFF76CFF5F
:10D388000DF107008DF80750FBF7CCF8FFF74AFFBF
:10D3980004469DF807003D70FBF7E8F82CB9347097
:10D3A800FFF76EFF0320FFF757FF204603B0F0BDDD
:10D3B8000824FAE72C46F8E7617F0020607F002008
:10D3C800054B1B7833B1054B1B780BB1FFF7C8BF72
:10D3D800FFF788BF08207047607F0020617F00202A
:10D3E800014B1878704700BF617F002007B50849D6
:10D3F8006846FBF743FC019B13B903B05DF804FBD7
:10D40800D3E9002090476846FBF742FCF3E700BFEA
:10D4180050DC0700FFF7EABF60DF704769DF70473D
:10D4280061DF704730B5114DADF5017D4FF4FA74E9
:10D438000DF1020103A8ADF80240FFF7F1FF70B942
:10D44800294601A8FBF71AFC029B002BF0D003A881
:10D45800D3E90021904701A8FBF71AFCF4E7052857
:10D4680001D0FCF75EFC0DF5017D30BD68DC0700DE
:10D47800024B1B780BB1FFF7D5BF7047637F0020C5
:10D4880018B1034B0360002070470E20704700BF9F
:10D4980068590020F0B5074685B00D4600295DD0D3
:10D4A8002F4B0B600C22002101A800F0E1F80126A7
:10D4B80006232A68ADF8083001A920208DF80470E9
:10D4C8008DF80660FFF7AAFF0C22002101A800F0E2
:10D4D800CFF800242A688DF8056001A94020ADF82E
:10D4E8000640FFF79BFF0C22214601A800F0C0F878
:10D4F800F7232A68ADF8063001A923208DF80470B7
:10D50800FFF78CFF0C22214601A800F0B1F82A6829
:10D518008DF8046001A93046FFF780FF0C222146F0
:10D5280001A800F0A5F84FF4B0632A68019301A997
:10D53800A120FFF773FF0C22214601A800F098F8FC
:10D548009DF804302A6864F3000301A9A0208DF82F
:10D558000430FFF763FF204605B0F0BD0E20FBE75F
:10D568006859002008B5FFF757FF10B9014B012291
:10D578001A7008BD637F00204BDF70471FB50D4C44
:10D5880001A8FFF7F9FF70B9214602A8FBF776FB5F
:10D59800039B002BF4D00198D3E90021904702A8FF
:10D5A800FBF776FBF4E7052801D0FCF7BAFB04B0DB
:10D5B80010BD00BF74DC07007AB370B414460F2A9C
:10D5C80015D902460B4640EA010515F0030F01D0B4
:10D5D800013C0EE0194610460432043306680D6813
:10D5E800AE4204D110461946043C042CF2D8013C42
:10D5F8000ED00A4603460444114618460133013248
:10D6080006780D78AE4203D118461146A342F3D1ED
:10D6180000780B78C01A70BC7047002070478446A9
:10D6280040EA010313F0030F18D18446202A0BD3D4
:10D638002DE9F007B1E8F807A0E8F807A2F1200201
:10D64800202AF7D2BDE8F007042A07D351F8043B93
:10D6580040F8043BA2F10402042AF7D2002A05D0BC
:10D6680011F8013B00F8013B013AF9D160467047D7
:10D678008446002A2DD010F0030F04D000F8011BB7
:10D68800013A26D0F7E7C9B241EA012141EA01414E
:10D69800202A12D3A2F120022DE9F0030B460C46F2
:10D6A8000D460E460F4688468946A0E8FA03203AFA
:10D6B800FBD2BDE8F00320320BD0042A05D340F892
:10D6C800041B043A05D0042AF9D200F8011B013AD8
:10D6D800FBD16046704700F1010110F0030F11D033
:10D6E80010F8012B002A23D010F0030F0AD010F8ED
:10D6F800012B002A1CD010F0030F03D010F8012BC7
:10D70800002A15D02DE970004FF001324FF0803318
:10D7180050F8044BA4EB020525EA04051D4000D18E
:10D72800F6E7A0F1040070BC10F8012B002AFBD129
:06D73800A0EB01007047A8
:08D7400085BF0700FDBC0700D6
:0CD74800000000000300000041D10700B9
:10D754003460002070700020817000203C60002044
:04D76400F4000000CD
:08D76800BDB90700000000003C
:08D77000E98907000000000038
:08D77800A98B0700000000006E
:10D7800079D407000000000085D5070000000000E4
:08D79000058B070000000000FA
:10D79800000000000000000075C007000010000035
:04D7A8000000080075
:10D7AC000010000004000000010000008188070048
:10D7BC00A5880700B588070025890700C5880700DC
:10D7CC008D880700918807009588070000100000DD
:10D7DC0004000000010000002D8A07000D8A0700DC
:10D7EC00FD890700358C0700E98B0700D1890700FC
:10D7FC00D5890700D9890700982F8A42914437713F
:10D80C00CFFBC0B5A5DBB5E95BC25639F111F159B7
:10D81C00A4823F92D55E1CAB98AA07D8015B8312F9
:10D82C00BE853124C37D0C55745DBE72FEB1DE80A5
:10D83C00A706DC9B74F19BC1C1699BE48647BEEFD4
:10D84C00C69DC10FCCA10C246F2CE92DAA84744A5F
:10D85C00DCA9B05CDA88F97652513E986DC631A8D5
:10D86C00C82703B0C77F59BFF30BE0C64791A7D5B4
:10D87C005163CA0667292914850AB72738211B2E3C
:10D88C00FC6D2C4D130D385354730A65BB0A6A7624
:10D89C002EC9C281852C7292A1E8BFA24B661AA830
:10D8AC00708B4BC2A3516CC719E892D1240699D640
:10D8BC0085350EF470A06A1016C1A419086C371EB9
:10D8CC004C774827B5BCB034B30C1C394AAAD84E97
:10D8DC004FCA9C5BF36F2E68EE828F746F63A578D2
:10D8EC001478C8840802C78CFAFFBE90EB6C50A465
:10D8FC00F7A3F9BEF27871C648002800002040005A
:10D90C0035AA0700D79307007B930700C39807003D
:10D91C003599070055990700C192070081920700BD
:10D92C0057980700000000001112131449878D331B
:10D93C00ACF07574A60E3A4CE29B9C8006FC8F6D85
:10D94C0085C96ECE99B9EF7B40424072984F8F4695
:10D95C00EC7667D7415F0A15BCE351C513E72193F9
:10D96C00ADF6E598C4737D48829CB84E0820000142
:10D97C00FFFFFFFFFFFFFFFFFFFFFFFF00000000A7
:10D98C00000000000000000001000000FFFFFFFF8E
:10D99C00512563FCC2CAB9F3849E17A7ADFAE6BC45
:10D9AC00FFFFFFFFFFFFFFFF00000000FFFFFFFF77
:10D9BC0096C298D84539A1F4A033EB2D817D03771D
:10D9CC00F240A463E5E6BCF847422CE1F2D1176BB8
:10D9DC00F551BF376840B6CBCE5E316B5733CE2B8B
:10D9EC00169E0F7C4AEBE78E9B7F1AFEE242E34FBA
:10D9FC004B60D2273E3CCE3BF6B053CCB0061D65F7
:10DA0C00BC86987655BDEBB3E7933AAAD835C65A7F
:10DA1C00DFA80700FDA3070059A4070000000000C1
:10DA2C00000000000338FDD8704700000101000021
:10DA3C00000101000000000027B8070021B8070012
:10DA4C0001B8070020000000780000000000000072
:10DA5C0001000100000000000100000000000000B7
:10DA6C000200050001000000420000000000000060
:10DA7C00000000000000000000000000000000009A
:10DA8C00010011000100FFFF010000000000000078
:10DA9C00020017000200FEFF64010000ECDA070030
:10DAAC00000000000000000000000000000000006A
:10DABC000100010000000000010000000000000057
:10DACC000200050001000000220000000000000020
:10DADC00000000000000000000000000000000003A
:10DAEC00010011000400FCFF040000000000000015
:10DAFC00020011000400FCFF040000000000000004
:10DB0C00030021000400FCFF0400100000000000D2
:10DB1C00040011000100FFFF0100000000000000E4
:10DB2C00050011000200FEFF0400000000000000D0
:10DB3C00060011000400FCFF0400000000000000BF
:10DB4C00070011000400FCFF0400000000000000AE
:10DB5C00080017000200FEFF24000000BCDA0700DA
:10DB6C00090010000100FFFF010000009CDB070012
:10DB7C000A0027000200FEFF440003005CDA0700E5
:10DB8C000000000000000000000000000000000089
:10DB9C0000000000010017000400FCFF68010000F9
:10DBAC008CDA0700020017000400FCFFAC01000037
:10DBBC00D0DB0700000000000000000000000000A7
:10DBCC0000000000010007000000000068010000D8
:10DBDC008CDA0700020001000000000001000000C8
:10DBEC0000000000030005000100000042000000DE
:10DBFC000000000000000000000000000000000019
:10DC0C0000000000446675546172670050EADA3017
:10DC1C008883B89F604F15F30000C98E0000000088
:10DC2C00000000000338FDD870470C000C00000009
:10DC3C00580201000007000070D7070078D70700D2
:10DC4C000800000080D7070090D7070008000000EC
:10DC5C0078D7070080D707000800000068D70700B6
:10DC6C0070D707000800000090D7070098D707006E
:04DC7C00080000009C
:10DC80000000000000000000000000000000000094
:10DC90000000000000000000000000000100000083
:10DCA0007C5900208C5900200090D003FF00FFFF1A
:08DCB0000100000000E0070084
:020000020000FC
:020000041000EA
:041014000080070051
:0410180000E00700ED
:040000037000835DA9
:00000001FF
